:100000004174731014802300040039280F0000018C
:100010000F0000018928F52801280F0000010F00BA
:1000200000016928FD20D5B7170500001305450F0D
:10003000970500009385C51393081008730000000E
:10004000170500001305E50D7300000017050000FB
:100050001305450D73000000170500001305A50CDE
:10006000730000008280170500001305650B9705DB
:1000700000009385650B93081008730000001705B6
:1000800000001305050A970500009385750A7300A3
:100090000000170500001305E5089705000093858B
:1000A000C50973000000170500001305C507970573
:1000B0000000938515097300000082801705000079
:1000C0001305050697050000938545089308100859
:1000D00073000000170500001305A5049705000034
:1000E000938555077300000017050000130585036D
:1000F000970500009385A506730000001705000012
:1001000013056502970500009385F505730000004F
:1001100082802F2004107300D000828031003200D2
:100120003300340052494E4720434C4F00524F4158
:10013000445345442000202020414E4F5254005447
:10014000202020482053540020464F4C2044455442
:10015000004C4F57204F55522000202020202020B7
:1001600020200020202020202020200020202020CF
:0601700020202020000009
:00000001FF
